:10000000830101308A001A29E20003088301DB0022
:100010000408DC000A08DD008A017008E3007108AA
:10002000E4007208E5007308E6007408E70075084C
:10003000E8007608E9007708EA007808EB0079081C
:10004000EC007A08ED007B08EE007C08EF005E080B
:10005000E0005F08E1008C1EF2281A088312A1005C
:1000600018128C122014DD22A422A208031D3F289E
:10007000A7010830A400A501A50A0430A3002208A6
:10008000033A031D4B289C21F0002106031D4B2839
:100090001530A200F228073022020318562801303A
:1000A0008A002208932121060319E4282208083A2D
:1000B000031D5E282108413A0319E4282208073A63
:1000C00003197A2809302202031C6A280E30220202
:1000D000031C7A2818302202031C72281D302202C9
:1000E000031C7A2822081E3A03197A282208203A8B
:1000F000031D832821080D3A0319F12821082C3A01
:10010000031DF228E42822080E3A031D9628210830
:100110000D3A0319F12821082C3A0319E42827087D
:10012000413E840021088000A70AF22822080F3AE5
:10013000031DA92821080D3A0319F12821082C3A9A
:100140000319E4282408413E840021088000A40A01
:10015000F2282208103A0319F12815302202031C54
:10016000BD28183022020318BD2801308A00220859
:10017000EC3E9B2121060319E42822081D3A031DA9
:10018000C5282108313A0319E42822081F3A031D23
:10019000D82821080D3A0319F12821082C3A03190F
:1001A000E42825084E3E840021088000A50AF22894
:1001B0002208213A031DED2821080D3A0319F128E0
:1001C00021082C3A031DE628A20AF22823084E3EF5
:1001D000840021088000A30AF2282208223A031989
:1001E000A014A20183126308F0006408F1006508FE
:1001F000F2006608F3006708F4006808F500690873
:10020000F6006A08F7006B08F8006C08F9006D0842
:10021000FA006E08FB006F08FC006008DE00610851
:10022000DF005C0884005D088A005B088300E20E42
:10023000620E0900203084002130302121308400FA
:100240004130302183010730DF00E630DE004130ED
:1002500084005B3034218301642C04068001840A0D
:100260000406031900342D29F0003F218000840A80
:10027000040870060319003435298312DE00DF1BE1
:1002800048295F088A005E08DE0A0319DF0A820037
:1002900083135F1883175E08DE0A840000080800D5
:1002A00048342E3447347234613466342034633435
:1002B00032343034303434340034573461346934B7
:1002C000743469346E346734203466346F34723475
:1002D00020340034733474347234653461346D34D2
:1002E0002E342E342E3420342034203400340D3477
:1002F0000A344334613472346D346F346E342034D4
:1003000044346934733470346C3461347934203457
:100310005634653472342E34203430342E34323432
:100320000D340A34003482072434473450345234B4
:100330004D3443342C3482074734473441342C3411
:10050C008312413423308312CE00080083168C16DC
:10051C000B178B17831208003330831699001815AC
:10052C001812831208008312BF003A303F020318DE
:10053C00A22A30303F020800031008003330831623
:10054C0099001815181283129817181683168C1602
:10055C008312080007309F00E03083168500831259
:10056C008501F73083168600831208008312AC00D5
:10057C000F30AC050508F039AD002C08AD042D0882
:10058C00850086150000000086110800D32A2B0870
:10059C0083122E23A90A0319AA0A83122A08DF0040
:1005AC0029083D21AB00AB0803190800CD2A8312A2
:1005BC00C0008316981CE02A831205088500981742
:1005CC0033308316990018151812981683124008A8
:1005DC00990008008312AA00AD01AD0AAE014423B4
:1005EC002A08F039F000F00E0F30F0057008AB005F
:1005FC00BC222A080F39AB00BC2A8312AB00AC001A
:10060C002A08DF002908A90A0319AA0A3D21F000CB
:10061C00AC0A2C038400700880008008031D062B94
:10062C002B0808008312A80020302802031C222B60
:10063C007F302802031C2A2B28080A3A03192A2B7C
:10064C0028080D3A031D2C2B031408000310080076
:10065C008312AC008316981C312B8312050885007D
:10066C0098173330831699001815181298168312A0
:10067C002C089900AD01AD0AAE01442B8312B001D8
:10068C00B101512BAF01AF0A73302F02031C492B60
:10069C00B00A0319B10A3108803AF0002E08803AEA
:1006AC007002031D5B2B2D08300283120318080007
:1006BC00482B8312A608031D652B7C306E2B260B52
:1006CC00692B2F306E2B2608023A031D702B2D3010
:1006DC00A900772B03302602031C772BA901FF30CE
:1006EC00A600A60A051200000000CB308312F022EF
:1006FC0005162908F02A8312A800A900AA011030B7
:10070C00F200F3012908F0002A08F100D32674083E
:10071C00A9007508AA00803AF000803070020A30F7
:10072C0003192902290803189D2B303E9E2B373EB6
:10073C0083122E230F30A8050A302802280803182C
:10074C00A92B303E2E2B373E2E2B8312A800A9004E
:10075C00AA011030F200F3012908F0002A08F10078
:10076C00D3267408A9007508AA00803AF0008030DE
:10077C0070020A300319290229080318C72B303ECE
:10078C00C82B373E8312DD220F30A8050A30280211
:10079C0028080318D32B303EDD2A373EDD2A1930CA
:1007AC008312AD00AE01442305120230F022193041
:1007BC00AD00AE0144230516A90100000000290874
:1007CC00413E84000008F022A90A0C302902031CC7
:1007DC00E32B051200000000C030F0220516A90121
:1007EC000000000029084E3E84000008F022A90AEF
:0407FC000C30290292
:1008000003180800F62B08308312AA002A08413E7C
:10081000840000082E3A0319122CAA0A0C302A026E
:10082000031C062C2A08A9000C30290203181F2CCF
:100830002908413E840020308000A90A142C2A088F
:10084000093A031D262C4908CB002E2C2A080A3A07
:10085000031D302C4A08CB004908CA002030C900CB
:10086000DF30CC00080004308312A90029084E3E76
:10087000840000082E3A0319422CA90A0A302902E2
:10088000031C362C2908073A0319612C2908053A5C
:10089000031D532C5408D6005208D4002E30D50026
:1008A0002030D300602C2908063A031D612C55081E
:1008B000D6005308D4005208D3002E30D500203083
:1008C000D2006D30D70008008312A010B02292220F
:1008D000A4227730A9000130AA00CC22BD24FA302E
:1008E000AD00AE014423D523A030AD000F30AE00E3
:1008F00044235030A9000130AA004E300323D523F1
:100900008830AD001330AE0044235D30A9000130C3
:10091000AA00413003236A30A9000130AA004E30FA
:100920000323D5238C22A0189C2C9030AD000130DD
:10093000AE0044235F23932CA01C9C2CA010831298
:10094000BA25032488223324D5235F23A80128084D
:10095000413E840020308000A80A0D302802031C8C
:10096000A72CA80128084E3E840020308000A80A49
:100970000D30280203189C2CB22C14308312AD00C9
:10098000AE01442305120330BC220530AD00AE0198
:1009900044230330BC22AD01AD0AAE014423033031
:1009A000BC220530AD00AE0144230230BC2205302C
:1009B000AD00AE0144232830F0220530AD00AE0179
:1009C00044230630F0220530AD00AE01442301304F
:1009D000F0220530AD00AE0144230C30F02205308A
:1009E000AD00AE0144234030F0220530AD00AE0131
:1009F000442305160030F0220530AD00AE0144233B
:100A00001030F0220530AD00AE0144230830F02252
:100A10000530AD00AE0144230430F0220530AD00B6
:100A2000AE0144230230F0220530AD00AE01442374
:100A30000130F0220530AD00AE0144230030F02239
:100A40000530AD00AE0144230030F0220530AD008A
:100A5000AE01442B2E2DB80A0319B90A83123908A6
:100A6000DF0038083D21203A03192B2D3908DF001B
:100A700038083D21093A03192B2DBB01BC01BD01EA
:100A8000BE01BA013908DF0038083D212D3A031DA7
:100A90004B2DBA0A522D3908DF0038083D212B3A78
:100AA000031D552DB80A0319B90A3908DF003808A3
:100AB0003D219922031C9A2D0A30F400F501F6011C
:100AC000F7013B08F0003C08F1003D08F2003E0849
:100AD000F300A9273908DF0038083D21DE00DF01D7
:100AE000D030DE070318DF0AFF30DF075E08F400AE
:100AF0005F08F500F601F70170087407F800750843
:100B0000F90071080318710FF9077608FA007208E6
:100B10000318720FFA077708FB0073080318730FA6
:100B2000FB077808BB007908BC007A08BD007B0889
:100B3000BE00522DBA080319B12D3B08F0003C0845
:100B4000F1003D08F2003E08F300F009F109F20956
:100B5000F309F00A0319F10A0319F20A0319F30A57
:100B600008003B08F0003C08F1003D08F2003E0898
:100B7000F30008008312A9012908413E84000008FF
:100B8000F0002908303E840070088000A90A073070
:100B90002902031CBC2DA9012908303E840000084D
:100BA0002E3A0319D82DA90A07302902031CCC2D8F
:100BB0000630290203180800290A303E8400000884
:100BC000F0002908303E840070088000A90A073030
:100BD00029020318F02D2908303E84002030E52D2D
:100BE000B7013030B8008030B90083122A25700870
:100BF000AC007108AD007208AE007308AF002C089D
:100C0000AA002D08AB00AC01AD01AE01AF01A901F6
:100C10002A08F0002B08F1000030F11BFF30F20031
:100C2000F3007008AC0771080318710FAD07720864
:100C30000318720FAE0773080318730AAF07A90AE7
:100C4000B9302902031C082E6430F400F501F601C6
:100C5000F7012C30840022278312B301B201B101C5
:100C6000B00100302F02031D3F2E00302E02031D65
:100C70003F2E03302D02031D3F2EE8302C02031CB3
:100C80006C2EB00A1830AC07FC3003110318013E7B
:100C9000031DAD07FF3003110318013E031DAE070E
:100CA000FF3003110318013E031DAF07312EB10AB7
:100CB0009C30AC07FF3003110318013E031DAD0744
:100CC000FF3003110318013E031DAE07FF3003116F
:100CD0000318013E031DAF0700302F02031D7A2EBB
:100CE00000302E02031D7A2E00302D02031D7A2EB5
:100CF00064302C02031C922E572EB20AF630AC0739
:100D0000FF3003110318013E031DAD07FF3003112F
:100D10000318013E031DAE07FF3003110318013E07
:100D2000031DAF0700302F02031DA02E00302E023E
:100D3000031DA02E00302D02031DA02E0A302C0210
:100D400003187D2EB008031DA82E2030B000AA2E57
:100D50003030B007B108031DB32E3008203A031D10
:100D6000B32E2030B52E3108303EB1003208303E6F
:100D7000B2002E30B3002C08303EB4006B30B5000A
:100D80006D30B600A9012908303E84000008F0004B
:100D90002908413E840070088000A90A0730290212
:100DA00003180800C32EF601F11FDD2EF009F00A2A
:100DB0000319F103F1097617F61773088039F6065F
:100DC000F31FE92EF209F20A0319F303F309E92EDE
:100DD000F601F401F50172087304031DF22EF0010F
:100DE000F10100341F30F6040310F60AF20DF30D82
:100DF000031CF52EF30CF20C73087102031D022F75
:100E000072087002031C0A2F7208F0027308031C98
:100E1000730AF102F40DF50DF60BF61AFA2EF61F11
:100E2000162FF409F40A0319F503F5097408F20002
:100E30007508F300761F0034F009F00A0319F10376
:100E4000F10900340008F000840A0008F100840A67
:100E50000008F200840A0008F3002F2F8401831297
:100E6000FC01F801F901FA01FB017408750476042C
:100E7000770403193E2FC030FC05492FF001F10122
:100E8000F201F301D72F0310F40DF50DF60DF70D58
:100E9000FC0AF71F432FFC0A0310F80DF90DFA0D99
:100EA000FB0D77087302031D5F2F76087202031D86
:100EB0005F2F75087102031D5F2F74087002031CF9
:100EC000712F78147408F0027508031C750FF10275
:100ED0007608031C760FF2027708031C770FF302E3
:100EE0000310F70CF60CF50CF40CFC037C083F39EE
:100EF000031D4C2F7C1F892F0310FF30F007F009D2
:100F0000031CF107F109031CF207F209031CF307A4
:100F1000F3097008F4007108F5007208F600730810
:100F2000F7007808F0007908F1007A08F2007B08F1
:100F3000F300FC1FD72F0310FF30F007F009031C4C
:100F4000F107F109031CF207F209031CF307F30987
:100F5000D72F84017008F8007108F9007208FA00B0
:100F60007308FB00F201F301F001F1010310FB0C27
:100F7000FA0CF90CF80C031CCB2F7408F007750859
:100F80000318750FF10776080318760FF207770834
:100F90000318770FF307780879047A047B040319A0
:100FA000D72F0310F40DF50DF60DF70DB62F8408AD
:100FB00003190034730880008403720880008403DE
:100FC0007108800084037008800000344334613469
:100FD00072346D346F346E34203444346934733475
:100FE0007034203400342D343E3456346534723439
:100FF0002E34203431342E34303420340034003454
:02400E00103F61
:00000001FF
